BL51 BANKED LINKER/LOCATER V5.03                                                        06/14/2006  17:38:47  PAGE 1


BL51 BANKED LINKER/LOCATER V5.03, INVOKED BY:
C:\KEIL\C51\BIN\BL51.EXE STARTUP.obj, main.obj TO buzzer RAMSIZE (256) CODE (0X0000-0X1FFF)


MEMORY MODEL: SMALL


INPUT MODULES INCLUDED:
  STARTUP.obj (?C_STARTUP)
  main.obj (MAIN)
  C:\KEIL\C51\LIB\C51S.LIB (?C?ULDIV)
  C:\KEIL\C51\LIB\C51S.LIB (?C?ULSHR)


LINK MAP OF MODULE:  buzzer (?C_STARTUP)


            TYPE    BASE      LENGTH    RELOCATION   SEGMENT NAME
            -----------------------------------------------------

            * * * * * * *   D A T A   M E M O R Y   * * * * * * *
            REG     0000H     0008H     ABSOLUTE     "REG BANK 0"
            DATA    0008H     0007H     UNIT         _DATA_GROUP_
            IDATA   000FH     0001H     UNIT         ?STACK

            * * * * * * *   C O D E   M E M O R Y   * * * * * * *
            CODE    0000H     0003H     ABSOLUTE     
                    0003H     0008H                  *** GAP ***
            CODE    000BH     0003H     ABSOLUTE     
                    000EH     07F2H                  *** GAP ***
            CODE    0800H     00E1H     UNIT         ?C?LIB_CODE
            CODE    08E1H     006CH     UNIT         ?PR?_TONEGEN?MAIN
            CODE    094DH     0048H     UNIT         ?PR?MAIN?MAIN
            CODE    0995H     0020H     UNIT         ?PR?_DELAYMS?MAIN
            CODE    09B5H     001BH     UNIT         ?PR?TMR0?MAIN
            CODE    09D0H     0011H     UNIT         ?PR?TMR0INIT?MAIN
            CODE    09E1H     000CH     UNIT         ?C_C51STARTUP



OVERLAY MAP OF MODULE:   buzzer (?C_STARTUP)


SEGMENT                          DATA_GROUP 
  +--> CALLED SEGMENT          START    LENGTH
----------------------------------------------
?C_C51STARTUP                  -----    -----
  +--> ?PR?MAIN?MAIN

?PR?MAIN?MAIN                  -----    -----
  +--> ?PR?TMR0INIT?MAIN
  +--> ?PR?_TONEGEN?MAIN

?PR?_TONEGEN?MAIN              0008H    0006H
  +--> ?PR?_DELAYMS?MAIN

*** NEW ROOT ***************************************************

BL51 BANKED LINKER/LOCATER V5.03                                                      06/14/2006  17:38:47  PAGE 2


?PR?TMR0?MAIN                  000EH    0001H



SYMBOL TABLE OF MODULE:  buzzer (?C_STARTUP)

  VALUE           TYPE          NAME
  ----------------------------------

  -------         MODULE        ?C_STARTUP
  C:09E1H         SEGMENT       ?C_C51STARTUP
  I:000FH         SEGMENT       ?STACK
  C:0000H         PUBLIC        ?C_STARTUP
  D:00E0H         SYMBOL        ACC
  D:00F0H         SYMBOL        B
  D:0083H         SYMBOL        DPH
  D:0082H         SYMBOL        DPL
  N:0000H         SYMBOL        IBPSTACK
  N:0100H         SYMBOL        IBPSTACKTOP
  N:0080H         SYMBOL        IDATALEN
  C:09E4H         SYMBOL        IDATALOOP
  N:0000H         SYMBOL        PBPSTACK
  N:0000H         SYMBOL        PBPSTACKTOP
  N:0000H         SYMBOL        PDATALEN
  N:0000H         SYMBOL        PDATASTART
  N:0000H         SYMBOL        PPAGE
  N:0000H         SYMBOL        PPAGEENABLE
  D:00A0H         SYMBOL        PPAGE_SFR
  D:0081H         SYMBOL        SP
  C:09E1H         SYMBOL        STARTUP1
  N:0000H         SYMBOL        XBPSTACK
  N:0000H         SYMBOL        XBPSTACKTOP
  N:0000H         SYMBOL        XDATALEN
  N:0000H         SYMBOL        XDATASTART
  C:0000H         LINE#         92
  C:09E1H         LINE#         99
  C:09E3H         LINE#         100
  C:09E4H         LINE#         101
  C:09E5H         LINE#         102
  C:09E7H         LINE#         151
  C:09EAH         LINE#         155
  -------         ENDMOD        ?C_STARTUP

  -------         MODULE        MAIN
  C:0000H         SYMBOL        _ICE_DUMMY_
  D:0090H         PUBLIC        P1
  D:00A0H         PUBLIC        P2
  B:00A8H.7       PUBLIC        EA
  C:0995H         PUBLIC        _DelayMs
  C:08E7H         PUBLIC        _ToneGen
  D:00CBH         PUBLIC        RCAP2H
  D:00CAH         PUBLIC        RCAP2L
  C:094DH         PUBLIC        main
  D:0089H         PUBLIC        TMOD
  B:00A8H.1       PUBLIC        ET0
  D:008CH         PUBLIC        TH0
  D:00CDH         PUBLIC        TH2
BL51 BANKED LINKER/LOCATER V5.03                                                      06/14/2006  17:38:47  PAGE 3


  D:008AH         PUBLIC        TL0
  D:00CCH         PUBLIC        TL2
  B:00A0H.0       PUBLIC        LED
  B:0088H.4       PUBLIC        TR0
  B:00C8H.2       PUBLIC        TR2
  C:09B5H         PUBLIC        Tmr0
  B:0090H.0       PUBLIC        BUZZER
  D:00C9H         PUBLIC        T2MOD
  D:00C8H         PUBLIC        T2CON
  C:09D0H         PUBLIC        Tmr0Init
  -------         PROC          TMR0
  -------         DO            
  D:000EH         SYMBOL        cnt
  -------         ENDDO         
  C:09B5H         LINE#         56
  C:09B9H         LINE#         59
  C:09BBH         LINE#         60
  C:09C5H         LINE#         61
  C:09C8H         LINE#         62
  C:09CBH         LINE#         64
  -------         ENDPROC       TMR0
  -------         PROC          TMR0INIT
  C:09D0H         LINE#         83
  C:09D0H         LINE#         84
  C:09D0H         LINE#         86
  C:09D3H         LINE#         87
  C:09D6H         LINE#         89
  C:09D9H         LINE#         90
  C:09DCH         LINE#         92
  C:09DEH         LINE#         93
  C:09E0H         LINE#         94
  -------         ENDPROC       TMR0INIT
  -------         PROC          L?0018
  -------         ENDPROC       L?0018
  -------         PROC          _TONEGEN
  D:0006H         SYMBOL        tone
  D:0008H         SYMBOL        duration
  -------         DO            
  D:000AH         SYMBOL        tmp
  -------         ENDDO         
  C:08E7H         LINE#         113
  C:08EBH         LINE#         114
  C:08EBH         LINE#         116
  C:08EFH         LINE#         117
  C:08EFH         LINE#         118
  C:08F2H         LINE#         120
  C:08F5H         LINE#         121
  C:08F8H         LINE#         123
  C:090FH         LINE#         124
  C:0925H         LINE#         125
  C:0933H         LINE#         126
  C:0939H         LINE#         127
  C:093CH         LINE#         128
  C:093FH         LINE#         130
  C:0941H         LINE#         131
  C:0948H         LINE#         132
  C:094AH         LINE#         133
BL51 BANKED LINKER/LOCATER V5.03                                                      06/14/2006  17:38:47  PAGE 4


  C:094AH         LINE#         134
  C:094CH         LINE#         135
  -------         ENDPROC       _TONEGEN
  -------         PROC          _DELAYMS
  D:0006H         SYMBOL        msec
  -------         DO            
  D:0004H         SYMBOL        x
  D:0002H         SYMBOL        y
  -------         ENDDO         
  C:0995H         LINE#         148
  C:0995H         LINE#         149
  C:0995H         LINE#         152
  C:099FH         LINE#         153
  C:099FH         LINE#         154
  C:09ADH         LINE#         155
  C:09B4H         LINE#         156
  -------         ENDPROC       _DELAYMS
  -------         PROC          MAIN
  C:094DH         LINE#         164
  C:094DH         LINE#         165
  C:094DH         LINE#         166
  C:0950H         LINE#         167
  C:0952H         LINE#         169
  C:0952H         LINE#         170
  C:0952H         LINE#         171
  C:0957H         LINE#         172
  C:095CH         LINE#         173
  C:0967H         LINE#         174
  C:0972H         LINE#         175
  C:097DH         LINE#         176
  C:0988H         LINE#         177
  C:0993H         LINE#         178
  -------         ENDPROC       MAIN
  -------         ENDMOD        MAIN

  -------         MODULE        ?C?ULDIV
  C:083CH         PUBLIC        ?C?ULDIV
  -------         ENDMOD        ?C?ULDIV

  -------         MODULE        ?C?ULSHR
  C:08CEH         PUBLIC        ?C?ULSHR
  -------         ENDMOD        ?C?ULSHR

******************************************************************************
* RESTRICTED VERSION WITH 0800H BYTE CODE SIZE LIMIT; USED: 0120H BYTE (14%) *
******************************************************************************

Program Size: data=16.0 xdata=0 code=499
LINK/LOCATE RUN COMPLETE.  0 WARNING(S),  0 ERROR(S)
